:100000000C94BA000C94D7000C94D7000C94D70031
:100010000C94D7000C94D7000C94D7000C94450393
:100020000C94D7000C9415030C94690D0C94D70014
:100030000C94D7000C94D7000C94D7000C94D700E4
:100040000C94D7000C94D7000C94D7000C94D700D4
:100050000C94D7000C94D7000C94D7000C94D700C4
:100060000C94D7000C94D700010A1003090309036C
:10007000090F14000F1400010203080A18030803F3
:1000800008001010202001010303080716030802CE
:10009000070010152525010104050C1025050C0588
:1000A0000C0C18000C1801010502070613020702C8
:1000B0000600101C283001010601023B59010227ED
:1000C0003B0205050B0B010007070B070B010101A4
:1000D000010207070D0D00000801040D19010407B6
:1000E0000E0005050F0F01000903060306010101BB
:1000F00001050D0D151500000C01023B59010227E9
:100100003B0206060C0C01000D081302050307084C
:10011000120000000A0A010000010203040506079C
:1001200008090A0B0C0D0E1013171B20262D364044
:100130004C5B6C8098B5D7FF807B130018001900CA
:100140000A000B0009001500000001001E0002005B
:1001500003000400050006000700520008001F000D
:1001600000001F0000001F1F1F1F000000000101F2
:100170000000093C11241FBECFEFD4E0DEBFCDBF8D
:1001800011E0A0E0B1E0E8E9F9E202C005900D92CB
:10019000AA34B107D9F712E0AAE4B1E001C01D9278
:1001A000AC33B107E1F70E947A0B0C94CA140C949B
:1001B0000000282F22952F709AE0299F900111248A
:1001C0008F70820F0895382F8DEC389FC001112455
:1001D000292F26952695269586EF9FEF289F802D1F
:1001E0001124830F2295207F822B0895FB01138217
:1001F00090E2918390836DEC869F90011124369557
:1002000036953695805D46EF5FEF349F902D112433
:10021000980F9283332381F0369FC0011124969565
:1002200096959695305D949F802D1124830F818340
:10023000992311F0905D90830895382FFB0112826D
:100240008DEC389FC0011124292F269526952695DF
:1002500011F480E202C0822F805D8083305D86EFE2
:100260009FEF289F802D1124830F81830895279865
:100270002F98549A5C988091FE018D7F10924E01C8
:1002800010924C0110924F0110924D0110925601A4
:1002900085608093FE0180E090E0FC01E45BFE4F0E
:1002A0001482019688309105C1F708952091FE01CE
:1002B00022FF6FC021FD57C01F9906C080915701D2
:1002C0008F5F8093570105C0809158018F5F8093A5
:1002D00058014091570130915801842F90E0830FCD
:1002E000911D843691050CF454C0442311F033233E
:1002F000C9F480914B018F5F80934B01843171F57C
:1003000010924B0180914A018F5F80934A011F9B9D
:1003100002C02F9801C02F9A8E3101F52F9A2260CA
:100320002B7F1AC080914B018F5F80934B018E31E0
:1003300021F426602093FE010895822F88703417DF
:1003400030F4882359F010924B01277F05C0882391
:1003500029F410924B0128602093FE01109257015E
:100360001092580108958091FD01882391F023FF98
:1003700003C01F9B0AC002C01F9907C080914C0197
:100380008F5F80934C015C98089521602093FE015B
:100390005C9A0895FC012091FE01822F85708530C2
:1003A00009F0E0C080914C01873008F4A7C080912B
:1003B0004C018E3428F480914C01803608F09EC0A8
:1003C00080914C018A3A20F080914D018A3321F4CA
:1003D00080914D018B33C0F010924E0110924C0170
:1003E00010924F0110924D011092560121602093FE
:1003F000FE0180E090E0FC01E45BFE4F1482019678
:1004000088309105C1F7A9C080914D01853108F46C
:1004100070C080914C018E3408F473C080914C01FF
:10042000803608F06EC080914C018735F0F48091E1
:100430004E018F5F80934E0180914D018C31A9F068
:1004400080914D01833289F0A0915601B0E0A45B08
:10045000BE4F14969C911497E0914F01F0E0E0504C
:10046000FF4F8081980F14969C9380914F018F5F6E
:1004700080934F0180914D018C3121F080914D018D
:100480008332E1F480914E0180FF18C010924E013A
:1004900010924C0110924F0110924D011092560192
:1004A00021602093FE0180E090E0FC01E45BFE4FC0
:1004B0001482019688309105C1F74FC080914D019B
:1004C0008C3181F080914D01833261F080914D013A
:1004D000893241F080914D018C3221F080914D01A3
:1004E000813339F4809156018F5F809356011092C9
:1004F0004F0180914D018F5F80934D0110924C010F
:100500002CC080914C018A3A40F180914C018B3B88
:1005100028F480914E018F5F80934E0180914D01B0
:100520008A3321F480914E0180FF2BC010924E013E
:1005300010924C0110924F0110924D0110925601F1
:1005400021602093FE0180E090E0FC01E45BFE4F1F
:100550001482019688309105C1F78091FE018E7F4B
:100560008093FE0180E00895FC01E45BFE4F14825D
:10057000019688309105C1F71092FD015C9881E0E9
:1005800008958091500184838091510183838091EB
:10059000520182838091530186838091540181832B
:1005A00080915501808310924E0110924C0110925F
:1005B0004F0110924D011092560121602093FE01CF
:1005C00080E090E0D1CF20916201309163014091B1
:1005D000640150916501211531054105510521F155
:1005E0008091FF01882301F580910801815080935B
:1005F00008018823C9F460915E0170915F018091C8
:100600006001909161016227732784279527609389
:100610005E0170935F0180936001909361010E947D
:10062000E30387E08093080108951F920F920FB6AD
:100630000F9211242F933F934F935F936F937F9368
:100640008F939F93AF93BF93EF93FF938091FF019D
:10065000882351F060915A0170915B0180915C0197
:1006600090915D010E94E303FF91EF91BF91AF91E3
:100670009F918F917F916F915F914F913F912F91BA
:100680000F900FBE0F901F9018951F920F920FB6EC
:100690000F9211242F933F934F935F936F937F9308
:1006A0008F939F93AF93BF93EF93FF938091FF013D
:1006B000882301F160915E0170915F01809160017A
:1006C000909161010E94E303809159018F5F8093B3
:1006D00059018F3079F4109259018091FF018150B6
:1006E0008093FF01E091FF01F0E0E85EFE4FE491AE
:1006F000E093B300FF91EF91BF91AF919F918F91E4
:100700007F916F915F914F913F912F910F900FBE0D
:100710000F901F90189526233723482359232093A1
:10072000620130936301409364015093650120910D
:100730005E0130915F014091600150916101209311
:100740005A0130935B0140935C0150935D016093CB
:100750005E0170935F01809360019093610110923C
:10076000FF010E94E3030895109262011092630159
:10077000109264011092650120915E0130915F0139
:10078000409160015091610120935A0130935B01C7
:1007900040935C0150935D010E94140460935E01DC
:1007A00070935F0180936001909361018FE180936A
:1007B000FF018091FF01E8E1F1E0E80FF11DE49114
:1007C000E093B3000895EF92FF920F931F937B0184
:1007D0008C010E94310D10FF02C0289A01C0289898
:1007E00011FF02C05F9A01C05F9812FF02C0429AD7
:1007F00001C0429813FF02C0439A01C043981F9161
:100800000F91FF90EF9008950E94460D209A579AFD
:100810003A9A3B9A28985F9842984398E0E7F0E02C
:100820008081836080830895CF92DF92EF92FF9260
:100830000F931F93CF93DF93FC01D3802481822FEA
:1008400065E00E947314392F822F0E947314C82E02
:10085000882331F4E12CF0ECFF2E012D112D27C05F
:1008600080913802C82FD0E08BE090E0C89FF00163
:10087000C99FF00DD89FF00D1124EF5DFE4FEC0DD8
:10088000F11D3197808190E0A0E0B0E08C01FF2461
:10089000EE2480E090E4A0E0B0E0E82AF92A0A2BF8
:1008A0001B2BCE5BDE4F8881C81608F0D394343002
:1008B00010F0A8E001C0A0E0333008F0A4603230AE
:1008C00008F0A2603111A1608D2D6CE00E947314BC
:1008D000E92FF0E0EE0FFF1FE75FFE4F808191816F
:1008E0009C0140E050E02E293F29402B512B8A2FBC
:1008F00090E0A0E0B0E0B82FAA2799278827282BFE
:10090000392B4A2B5B2B91E0D91619F0ADE0DA16A2
:1009100019F4CC2009F4277FB901CA01DF91CF91E6
:100920001F910F91FF90EF90DF90CF9008958091ED
:100930006601882341F41092B90080E28093B800E8
:1009400081E08093660180E00895982FFB0184EA9E
:100950008093BC008091BC0087FFFCCF8091B900E0
:10096000887F883011F0803181F49093BB0084E857
:100970008093BC008091BC0087FFFCCF8091B900C0
:10098000887F883129F0803419F0808381E00895D0
:1009900080E00895982F44EA34E824E94093BC00AD
:1009A0008091BC0087FFFCCF8091B900887F8830A0
:1009B00011F0803199F79093BB003093BC00809187
:1009C000BC0087FFFCCF8091B900887F803211F096
:1009D000883539F42093BC008091BC0084FDFCCFA5
:1009E000DDCF08950E94A504089584E98093BC009A
:1009F0008091BC0084FDFCCF0895FB018093BB0077
:100A000084E88093BC008091BC0087FFFCCF80917C
:100A1000B900887F883211F480E00895808381E0F6
:100A2000089584EC8093BC008091BC0087FFFCCFCC
:100A30008091BB00089584E88093BC008091BC0045
:100A400087FFFCCF8091BB000895809168010895D5
:100A5000EF92FF920F931F93CF93DF93182FF62EF1
:100A6000E72E042F80916701882391F1442381F1BF
:100A7000812F90E0840F911D813491054CF580ED1C
:100A80000E94CA04812F68E671E00E94FD04882359
:100A9000D9F481ED68E671E00E94F2048823A1F4A4
:100AA000CF2DDE2D102F7E0105C00E941105F7010C
:100AB00081937F011150C9F70E941B050150C00F9F
:100AC000D11D888311E001C010E00E94F50401C02F
:100AD00010E0812FDF91CF911F910F91FF90EF9048
:100AE0000895EF92FF920F931F93CF93DF93082FF8
:100AF000F62EE72E142F80916701882341F14423BD
:100B000031F1802F90E0840F911D81349105FCF428
:100B100080ED0E94CA04802F68E671E00E94FD0407
:100B2000882389F48F2D9E2D9C01E901888168E638
:100B300071E00E94FD041150882329F421961123AD
:100B4000A9F711E001C010E00E94F50401C010E017
:100B5000812FDF91CF911F910F91FF90EF9008951A
:100B6000EF92FF920F931F93DF93CF9300D0CDB7F7
:100B7000DEB78C017B018FEFFB0180830E9497041D
:100B8000F80180838823C9F481E08093670180E8BD
:100B900080936901809169018A8387E0BE016E5F5D
:100BA0007F4F41E00E9471058823E9F483E0F8015A
:100BB000808380916801F701808380E00BC0898188
:100BC00087FF07C08F77898380E0B80141E00E94EA
:100BD000710581E00F900F90CF91DF911F910F91E0
:100BE000FF90EF90089580E08E010F5F1F4FB801D6
:100BF00041E00E942805882311F7EBCF0F931F9344
:100C0000DF93CF93CDB7DEB727970FB6F894DEBF4B
:100C10000FBECDBF8C0180916701882379F180E000
:100C2000BE016F5F7F4F47E00E942805882331F1A6
:100C30008F810E94D900F80180838E810E94D900A3
:100C4000F80181838D810E94D900F80182838C8113
:100C50000E94D9008150F80186838B810E94D900BF
:100C6000F80183838A810E94D900F80184838981F5
:100C70000E94D900F801858381E001C080E02796B9
:100C80000FB6F894DEBF0FBECDBFCF91DF911F919D
:100C90000F9108950F931F93DF93CF93CDB7DEB7D6
:100CA00027970FB6F894DEBF0FBECDBF8C018091A1
:100CB0006701882369F1F80185810E94E300898337
:100CC000F80184810E94E3008A83F80183810E94F5
:100CD000E3008B83F80186810E94E3008F5F8C83A1
:100CE000F80182810E94E3008D83F80181810E94D6
:100CF000E3008E83F80180810E94E3008F8380E00F
:100D0000BE016F5F7F4F47E00E947105811181E056
:100D100027960FB6F894DEBF0FBECDBFCF91DF91FF
:100D20001F910F9108952E9826980895FC018091A7
:100D30008B01882309F473C080918C01823051F1BA
:100D4000833009F04BC020918F0130919001809148
:100D50008F0190919001232F33278095909590706B
:100D60002817390709F058C080918F0190919001A0
:100D700090709093900180938F0120918F0130911A
:100D800090018091910190919201982F8827822B58
:100D9000932B20C020918F013091900180918F0181
:100DA00090919001232F332780959095907028176C
:100DB000390759F080918F01909190018070805097
:100DC000914D51F58BE080938C0180918F01909132
:100DD000900190709093900180938F0180918C018D
:100DE000808380918D0190918E0192838183809187
:100DF0008F019091900194838383809193018583E7
:100E00001092900110928F0110928E0110928D011C
:100E10001092930181E001C080E010928B0108954F
:100E2000982F60917A0170918401671738F1809151
:100E30008501681718F580918A01292F30E04091CB
:100E4000940150919501882381F0862F90E0871BB3
:100E5000910902C0220F331F8A95E2F7422B532BD0
:100E6000509395014093940151C0440F551F242B7A
:100E7000352B309395012093940148C070918601E1
:100E8000671738F180918701681718F580918A01FA
:100E9000292F30E04091960150919701882381F0ED
:100EA000862F90E0871B910902C0220F331F8A957D
:100EB000E2F7422B532B509397014093960126C0A3
:100EC000440F551F242B352B309397012093960107
:100ED0001DC080917B018330C9F46131B8F0653168
:100EE000A8F4892F90E0262F30E02151304002C035
:100EF000880F991F2A95E2F7209198013091990166
:100F0000282B392B30939901209398016F5F6093C0
:100F10007A01089593B180918B01882309F06DC304
:100F2000292F207480917901882359F590917601B9
:100F3000222321F49F5F9093760108959923B9F0BD
:100F400091E090937901909377011092780110923B
:100F500097011092960110929501109294018FEFD3
:100F600080937A019093750110926C01089580919D
:100F70006F019091700101969093700180936F01C1
:100F8000089580917701882309F40FC1222349F045
:100F9000809175018F5F80937501893708F450C285
:100FA0006EC120917601822F8651883058F480914D
:100FB0007501833038F0883028F48BE791E068E6DB
:100FC00070E02FC0822F86538934E8F48091750138
:100FD0008D508333C0F48BE791E068E770E040E127
:100FE00050E00E944E1480917501803208F0B9C023
:100FF000109284011092850110928601109287014F
:1010000010928801AEC0822F8452833178F480918F
:101010007501843258F0873348F48BE791E068E833
:1010200070E040E150E00E944E149BC0822F8C5132
:101030008F3058F4809175018C3138F08B3228F460
:101040008BE791E068E970E0ECCF822F8851853121
:1010500058F4809175018C3038F0873128F48BE793
:1010600091E068EA70E0DDCF322F3150323058F431
:10107000809175018B3338F08A3528F48BE791E045
:1010800068EB70E0CECF822F8750853018F0875004
:10109000893038F590917501892F8750853018F087
:1010A0009E509930F0F48BE791E068EC70E040E1FD
:1010B00050E00E944E149091750190936B018091C5
:1010C00076018C508B3018F09C509B3030F410928D
:1010D0006A0180E480936C0144C081E080936A01DE
:1010E00040C0343050F4809175018750833128F42A
:1010F0008BE791E068ED70E094CF822F83518131CE
:1011000098F480917501863078F08D3068F48BE723
:1011100091E068EE70E040E150E00E944E141092C1
:101120006B0110926A011DC0323058F48091750134
:101130008D3138F08D3228F48BE791E068EF70E064
:1011400070CF28502C3058F480917501823038F0DF
:10115000863028F48BE791E068E071E062CF10926E
:10116000790110927A0180917B01873051F480914E
:1011700075018C508B3060F080916A01882369F48E
:101180000AC0883051F4809175018D508D3010F473
:1011900081E001C080E00E94100781E08093760129
:1011A00010927501109277014BC1809178018823CC
:1011B00009F439C1222309F469C040917A01609190
:1011C0008801461799F480918901813079F49091D2
:1011D000760180918001981708F451C080918101B7
:1011E000891708F44CC0109289012AC150917501E9
:1011F0005F5F5093750180917B01813091F45A308B
:1012000058F14B3048F14F5F409388014150809135
:101210008601480F4F5F4093870188E080937501F6
:1012200035C0873029F45731B8F04B30A8F00CC0E6
:10123000893091F45D3080F0242F30E0862F90E0EB
:1012400002972817390744F080918901882321F4F7
:1012500081E0809389011AC0593708F4F1C0242F26
:1012600030E0862F90E001972817390741F48091EC
:101270008901882321F44F5F40937A01E1C01092E5
:1012800079011092760110927501DAC080917B018C
:101290008730F1F4809176018C508B3048F481E0F6
:1012A0000E94100780E00E94100710926A0150C04F
:1012B00080916B018C5090916A018B3038F480E002
:1012C000992309F481E080936A0140C0892F3EC0D0
:1012D000893009F042C030917A01832F8350909178
:1012E0007601833078F49C3038F0809175018C3031
:1012F00018F081E00E94100780E00E941007109211
:101300006A0174C09750963050F480E00E94100734
:1013100081E00E94100781E080936A0119C08091EA
:101320006B01875090916A01863038F420E0992350
:1013300009F421E020936A0101C0292F313029F4FA
:10134000222319F484E280938801822F0E941007DF
:101350008091750180936B0149C0833081F5809144
:101360007A01803161F5809176018350863008F0F2
:1013700054C080917501843260F0873350F410922C
:101380007801109299011092980181E180937A017D
:1013900048C08750803110F481E001C080E00E9495
:1013A0001007109278018AE080937B0180E180939E
:1013B000860180E2809387018093880132C09091FA
:1013C000760180917C019817A0F080917D018917AA
:1013D00080F02091750180917E01281750F0809156
:1013E0007F01821730F081E00E941007109278018F
:1013F00018C080918001981780F080918101891731
:1014000060F09091750180918201981730F0809181
:101410008301891710F080E0E7CF109279011092D4
:10142000750181E005C0222331F4809176018F5F40
:101430008093760105C081E08093780180937501E7
:1014400040917A0180918801481709F0D6C08091B7
:101450008901882309F0D1C060917B01613021F0BE
:101460006A3011F06D30B9F4209171013091720140
:1014700080919601909197012817390761F4809126
:101480006F0190917001845F914028F41092700177
:1014900010926F016EC081E080938B01683049F536
:1014A00040919601509197019A01209530953370A3
:1014B00080916D0190916E012817390799F430934E
:1014C00097012093960160938C01809194019091F3
:1014D000950190938E0180938D013093900120931C
:1014E0008F0147C010928B0150936E0140936D01A4
:1014F00040C06230B9F44423A9F480917301909103
:101500007401909395018093940180917101909161
:10151000720190939701809396018091930181606D
:101520008093930160938C01809194019091950137
:1015300090938E0180938D01909374018093730139
:1015400080916C0190E02091960130919701822B5F
:10155000932B9093970180939601909390018093A1
:101560008F018091980190919901909392018093BD
:10157000910180918B018823B1F120918F013091ED
:101580009001809171019091720182179307B9F4D3
:1015900020918D0130918E018091730190917401A1
:1015A0008217930761F480916F0190917001885EBA
:1015B000934028F4809193018160809393018091FE
:1015C000940190919501909374018093730180919F
:1015D00096019091970190937201809371011092FE
:1015E000700110926F011092790110929701109280
:1015F000960110927601109275010895DF93CF93B2
:101600000F92CDB7DEB780E680937C0085E88093AB
:101610007A0080917A00806480937A0080917A00C9
:1016200086FDFCCF80917900898320E030E08981BC
:10163000F901E556FE4F80832F5F3F4F2031310582
:10164000B1F7898190E09093AC018093AB018091D8
:10165000AB019091AC0124E0880F991F2A95E1F726
:101660009093AC018093AB0180917A008064809369
:101670007A000F90CF91DF9108958091AB01909106
:10168000AC0134E0969587953A95E1F780950895F9
:1016900080917A0086FD27C0409179008091AB014E
:1016A0009091AC0130919A01E32FF0E0E556FE4FA6
:1016B0002081821B91099093AC018093AB01408300
:1016C0008091AB019091AC01840F911D9093AC017E
:1016D0008093AB013F5F3F7030939A0180917A0015
:1016E000806480937A0008958091B5018F5F809324
:1016F000B50108951F93DF93CF9300D0CDB7DEB728
:101700000E94C80D0E94C4130E9437010E94040465
:10171000CE010196BE016E5F7F4F0E94B0050E9410
:10172000FE0A0E949A0C0E9493060E94590D0E9484
:101730002F0F78940E941C0C8FE10E94E70C11E09F
:101740000E943D0B982F9695969596958091450110
:10175000891711F0909345019091B5018091460150
:10176000891709F453C09091B5018091B40198177D
:1017700040F08DEA91E00E94FE05882309F446C0FE
:1017800004C08091B5018093B2019091470180918E
:10179000B101981791F08DEA91E00E94911080912B
:1017A000B101809347019091B00180914801891760
:1017B00021F01093FD0190934801809146018F3FE5
:1017C00051F08091B5012091B201281720F4909139
:1017D000B501921B01C090E08091B2018093B501E8
:1017E0008091B50180934601992329F08091B5013C
:1017F000815F891B03C08091B501815F8093B40133
:101800008091B4018C3310F01092B4010E94061143
:101810008DEA91E00E94CA01882309F491CF8DEAF4
:1018200091E00E944A068091B2018093B5018DEA51
:1018300091E00E94911084CF84B5806884BD84B506
:10184000806284BDE0EBF0E080818062808381E093
:101850008093B60108955E9884B58F7784BD5D98B6
:1018600084B58F7D84BD5B98E0EBF0E080818F7D57
:1018700080831092B60108952091B80130E02F5F67
:101880003F4F8093BD016093BE014093BF0190E044
:10189000FC01E29FC001E39F900DF29F900D112487
:1018A00097BD70E0629FC001639F900D729F900D85
:1018B000112498BD50E0429FC001439F900D529F5C
:1018C000900D11249093B40008958091B90188235C
:1018D00081F4E09139028091B701E80FE7FDE0E083
:1018E000EF71FF27E7FDF095E85EFE4FE491E0938E
:1018F000B8018091BD016091BE014091BF010E947D
:101900003C0C08958091B601882319F00E942B0C9D
:10191000089584B5806884BD84B5806284BD80915B
:10192000B00080628093B00081E08093B6010E9495
:10193000650C08955E98569A83E084BD85BD8093BA
:10194000B00084E08093B1005D98559A5B98539AFB
:101950000E94650C0895FC01DB018091BD0180832C
:101960008091BE018C938091BF01FA01808308951C
:10197000803208F08FE1603208F06FE1403208F009
:101980004FE18093BA016093BB014093BC01E82F03
:10199000F0E0E85EFE4F8491E62FF0E0E85EFE4F57
:1019A0006491E42FF0E0E85EFE4FE4914E2F0E9438
:1019B0003C0C0895FC01DB018091BA018083809189
:1019C000BB018C938091BC01FA0180830895982F0C
:1019D0008091B601882351F0903220F08FE18093FE
:1019E000B70102C09093B7010E94650C08958091E1
:1019F000B601882389F030913902832F992787FD1A
:101A000090952091B701820F911D4F972CF43F5F65
:101A1000309339020E94650C08958091B6018823A5
:101A200091F030913902832F992787FD909520916D
:101A3000B701820F911D181619062CF431503093FE
:101A400039020E94650C089591E09093B90180934A
:101A5000B8010E94650C08951092B9010E94650CAE
:101A600008959B01AC01BB27A52F942F832F9EBD0A
:101A70000DB407FEFDCF8EBD0DB407FEFDCF2EBD0C
:101A80000DB407FEFDCF2A982A9A089584B18C627E
:101A900084B9249885B1846185B988E58CBD8DB5FC
:101AA00081608DBD60E070E080E090E00E94310DCB
:101AB00008958FE193E0909387008093860082E001
:101AC0008093800089E18093810080E280936F00A1
:101AD00008951F920F920FB60F9211242F933F93E8
:101AE0004F935F936F937F938F939F93AF93BF9326
:101AF000EF93FF930E948A078091C4018F5F8093C8
:101B0000C4018A30A1F51092C4018091C3018F5F96
:101B10008093C3018A3059F51092C3010E94560187
:101B20000E9470108091C2018F5F8093C2018A3041
:101B3000F1F41092C2010E945E100E94E3028091B3
:101B4000C1018F5F8093C1018A3089F41092C10175
:101B50000E94740B0E94480B0E94BF0F8091C0012D
:101B60008F5F8093C0018C3311F41092C001FF91FC
:101B7000EF91BF91AF919F918F917F916F915F9105
:101B80004F913F912F910F900FBE0F901F9018957E
:101B9000E1ECF0E08081886080831092C50083E3EF
:101BA0008093C4000895982F8091C00085FFFCCFDA
:101BB0009093C6000895FC0107C08091C00085FF86
:101BC000FCCF31969093C60090819923B1F7089588
:101BD0009C0106C08091C00085FFFCCF9093C60099
:101BE000F9012F5F3F4F94919923A1F70895FF9238
:101BF0000F931F93CF93DF93F82E1091D8011150BC
:101C00005091F4014091F2013091F101C12FDD2793
:101C1000C7FDD095CB53DE4F212FFE0101E061E0DF
:101C20001AC08081813011F4952F09C0863011F4DB
:101C3000942F05C0853011F090E001C0932F002350
:101C400019F480E090E004C080E0911181E08627E3
:101C5000082F215031972F1524F7002369F40EC067
:101C60008881843011F40E942C0D8091D80181501C
:101C70008093D801115021971F1594F7802FDF9181
:101C8000CF911F910F91FF900895EF92FF920F93C4
:101C90001F937A018B010E941404A80197010E94EE
:101CA0008B031F910F91FF90EF9008950F931F9357
:101CB0008C018091E60190E0FC01EE0FFF1FE80F20
:101CC000F91FE050FE4F86A167A140A50E94B80C05
:101CD000012B49F44091E60150E04F5F5F4F81E0F6
:101CE00068E00E940D0F1F910F910895DF93CF932D
:101CF000CDB7DEB727970FB6F894DEBF0FBECDBFC6
:101D0000982F8091D801E82FFF27E7FDF095EB533E
:101D1000FE4F9083E92FF0E0E153FE4F80838F5F09
:101D20008093D801973001F5A5EFB1E0FB0187E082
:101D300001900D928150E1F71092FC0181E08093B7
:101D4000F4018091F80188508C3010F48FEF01C0BD
:101D500084E60E94240D85EF91E04FEF5FE360E0A1
:101D600070E00E94450E50C0913021F4CB010E94DA
:101D7000560E4AC09630C1F4FE01319687E0DF016D
:101D80001D928A95E9F7809132028C83809133020B
:101D90008D831092F30186E067E0AF010E940D0F82
:101DA00081E08093F20130C0953051F485E067E026
:101DB0004CED51E00E940D0F81E08093F10124C0B1
:101DC0009830B1F48AE08093E501862F6CE00E94A0
:101DD0007314E92FF0E0EE0FFF1FE75FFE4F608105
:101DE000718180E090E020E030E040E050E00AC007
:101DF000992351F460E070E080E09FE020E030E063
:101E000040E05FE00E948B0327960FB6F894DEBF98
:101E10000FBECDBFCF91DF9108951F93CF93DF9376
:101E2000162FEA018F3F11F4E0E008C0E82FFF27EA
:101E3000E7FDF095E153FE4FE081EF5F8091D8011F
:101E4000E81729F08E2F0E94F70D882321F0812FAB
:101E5000BE010E94760EDF91CF911F91089581E01F
:101E600061E070E00E94760E80E060E070E00E9429
:101E7000760E399A219A0895EF92FF920F931F934D
:101E8000DF93CF93CDB7DEB727970FB6F894DEBFB9
:101E90000FBECDBFF82E8B01EF2DF0E0E153FE4FCA
:101EA000E0808E2D0E94F70D8CED91E040E050E037
:101EB00060E070E00E94450EEE2DFF27E7FDF095F3
:101EC000EC53FE4F80818630B1F587E0F81609F0BB
:101ED00049C0DE011196F80101900D928150E1F7A1
:101EE0009091F301E92FF0E0EE0FFF1FE050FE4F5D
:101EF0008C8182AB8D8183AB9F5F9093F301923095
:101F000041F41092F20186E060E070E00E943C0F24
:101F100029C0E92FF0E0EE0FFF1FE050FE4F82A92D
:101F20008C8383A98D8386E067E0AE014F5F5F4FAE
:101F30000E940D0F17C08530A9F487E0F81691F4C0
:101F4000C8010E944A06ACEDB1E0F80187E00190BB
:101F50000D928150E1F71092F10145E0F42E00E07E
:101F600010E09ACF27960FB6F894DEBF0FBECDBF14
:101F7000CF91DF911F910F91FF90EF900895E09125
:101F8000D801FF27E7FDF095EC53FE4F80818823B1
:101F900071F48091E3018F3F51F08F5F8093E301F3
:101FA000873029F480E060E070E00E943C0F80916F
:101FB000DB01893718F48F5F8093DB018091DB01AF
:101FC000883729F480E092E06CE30E949E13089524
:101FD000DF93CF9300D00F92CDB7DEB7823021F5DB
:101FE0008091F0018F5F8093F001853008F460C02C
:101FF00061E070E080E090E00090EF0104C0660FC7
:10200000771F881F991F0A94D2F720E030E040E044
:1020100050E00E948B038091EF018F5F8F7180935E
:10202000EF011092F00144C0883069F48091E5011D
:1020300081508093E5018823D9F588E060E070E065
:102040000E943C0F35C0843049F4E091D301F0E0A8
:10205000EC53FE4F80810E94E80F2AC0833041F587
:102060008091EE018F5F8093EE0190913702891786
:10207000F8F08091EC019091ED01019661E076E03D
:102080000E947F148093EC019093ED01BE016F5F7D
:102090007F4FAE014E5F5F4F9E012D5F3F4F0E940D
:1020A000DF1389816A814B810E943C0C1092EE0102
:1020B0000F900F900F90CF91DF910895E091D8018C
:1020C000FF27E7FDF095EC53FE4F80810E94E80F5B
:1020D0008091D901882319F081508093D901089506
:1020E000E091D801FF27E7FDF095EC53FE4F80818A
:1020F0008430B1F48091EB018F5F8093EB0190917C
:102100003602891768F08091EA010E9436140E9415
:10211000240D8091EA018F5F8093EA011092EB0118
:102120000895009709F45BC0ACEDB1E0FC0187E0D5
:1021300001900D928150E1F78091DB01883708F41E
:102140004EC08091DA01882309F049C02091DF0157
:102150007091E0015091320230913302409134028B
:10216000E0913502521748F0251719F080E090E011
:1021700006C080E090E0731710F081E090E0682FD7
:10218000241718F421E030E00CC0241719F020E0E7
:1021900030E007C080E090E07E1710F481E090E02E
:1021A0009C01451748F4662321F480E090E0222347
:1021B00079F081E090E00CC0662319F480E090E0B3
:1021C00007C090E0222309F491E081E09827892F4D
:1021D000882319F40E941C0C02C00E942B0CE09171
:1021E000D801FF27E7FDF095EC53FE4FE081EE2389
:1021F00061F0E83051F0E23041F0E53031F0E630A6
:1022000021F08CED91E00E94B40308952F923F924B
:102210004F925F926F927F928F929F92AF92BF92F6
:10222000CF92DF92EF92FF920F931F93DF93CF93A2
:10223000CDB7DEB729970FB6F894DEBF0FBECDBF7E
:10224000CE0104960E949606882309F456C2809116
:10225000D901882309F051C283E08093D9014091CC
:10226000D801E42FFF27E7FDF095EC53FE4F808166
:10227000882309F047C02091E4014D815E8122232B
:1022800011F180910002909101028417950729F5C0
:10229000E22FF0E0EE0FFF1FE050FE4F8F81988598
:1022A00091838083223159F480E092E068E30E94B8
:1022B0009E1380E060E070E00E943C0F1EC22F5F22
:1022C0002093E4010AC08FEF8093E3015093010251
:1022D0004093000281E08093E4018091E4016CE08E
:1022E0000E947314E92FF0E0EE0FFF1FE75FFE4F2F
:1022F0002081318140E050E05F60CA01B9010E9455
:102300008B03FBC120910002309101028D819E81DF
:102310002817390709F0F1C12F813885E2E0F2E092
:1023200010E004C01F5F3296123191F080819181DC
:1023300082179307B9F7112359F490E08091DA01DD
:10234000882309F491E09093DA010E94820CC6C1BF
:10235000D42EDA94ED2CFF24E7FCF09485EC91E088
:10236000E80EF91E80E0012F035092E0492E512C17
:102370004C0E5D1EB3E08B2E912C8C0E9D1E3E01EB
:102380000894611C711CAAE0CA2EA12CF6E0BF2E95
:10239000E4E03E2E72E0272E39C1F70180818730BC
:1023A00009F085C0E091D601F0E0EC53FE4FE081EA
:1023B000E53019F41530E1F404C0E630C9F4163004
:1023C000B9F48091FC01882321F4F1E0F093FC0141
:1023D0005CC0813009F059C01092FA011092F401EA
:1023E0000E942C0D87E065EF71E00E943C0F05C153
:1023F000023008F04AC0133011F04FEF01C041E045
:102400008091FC018823F1F44F3F41F48091F80161
:10241000882321F437E13093F80109C08091F80155
:10242000840F8093F801883110F01092F8018091A8
:10243000F80188508C3010F48FEF01C084E60E94C0
:10244000240D23C0813009F5E63019F44C9D402D50
:10245000112447FF11C02091F90130E0842F992702
:1024600087FD9095909581959F4F2817390724F403
:10247000445C4093F90109C08091F901840F809375
:10248000F9018C3310F01092F9018091FC0188233E
:1024900029F040E050E06FEF7FE004C04FEF5FE3D2
:1024A00060E070E085EF91E00E94450EA6C08130AB
:1024B00009F082C0183059F48091E6018F5F837073
:1024C0008093E60180E090E00E94560E96C01C309A
:1024D00019F41092E70191C01D3019F48093E701BF
:1024E0008CC01E3019F42092E70187C01F3019F408
:1024F0003092E70182C0023008F082C0133011F040
:102500002FEF01C021E09091E7019430E8F4809131
:10251000E60133E0839FF0011124EA5DFD4FDF0106
:10252000A90FB11D8C912F3F29F4882339F08150D8
:102530008C9304C08F3110F4280F2C93808161811B
:1025400042810E94B80C59C02F3F59F48091E80194
:102550009091E9010A9798F4B092E901A092E801FC
:102560001CC0213061F48091E8019091E901865FFF
:10257000954028F01092E9011092E8010EC0FC2D60
:102580002F02C00111242091E8013091E901820F4E
:10259000931F9093E9018093E8018091E801909165
:1025A000E901B301A20194010E94DF1389816A81CC
:1025B0004B810E943C0C21C0843079F4023000F53C
:1025C000133009F08EC0809136028230B0F0815015
:1025D00001C08F5F8093360210C0833089F40230CF
:1025E00078F4133009F083C080913702823028F0EC
:1025F000815001C08F5F8093370281E090E002C07C
:1026000080E090E0DA940894E108F108D7FC04C077
:10261000882309F4C2CE62C0882309F05FC011305C
:1026200019F40E94F70C5AC0123019F40E940D0DD3
:1026300055C0183019F48FEF61E042C0153011F425
:1026400085E003C0163031F486E060E070E00E945F
:10265000760E44C01B3019F48FEF62E031C01930A0
:10266000A9F48091D801E82FFF27E7FDF095EC53FE
:10267000FE4FE081E43021F481500E94F70D2EC01E
:10268000E13011F0E33051F584E0DFCF1131A1F4F6
:10269000809138028F5F63E00E947314692F9093DA
:1026A000380270E06F5F7F4F88E00E94760E80E016
:1026B00090E00E94911012C01A3039F48FEF63E05D
:1026C00040E050E00E940D0F09C0173021F481E076
:1026D0008093FD0103C0103181F4319A1092DB0127
:1026E0000CC080913602853008F473CF86CF80917C
:1026F0003702883008F47ECF80CF29960FB6F89441
:10270000DEBF0FBECDBFCF91DF911F910F91FF9024
:10271000EF90DF90CF90BF90AF909F908F907F9081
:102720006F905F904F903F902F9008959C01F99982
:10273000FECF32BD21BDF89A80B5089520E032E089
:10274000982F921B6150690F1CC0E92FF0E0F99996
:10275000FECF9F012050304032BD21BDF89A80B598
:10276000E050FE4F4081841759F0F999FECF1FBA0F
:1027700032BD21BD40BD0FB6F894FA9AF99A0FBE4A
:102780009F5F691710F7089580E092E060E070E0C5
:102790004CE350E026E933E10E94571480913A025D
:1027A000893021F480913B028C3341F080E092E04B
:1027B00068E371E04CE350E00E944E140895CF931B
:1027C000DF93EB01FA01D9019C0120503C4FAC0191
:1027D00040505E4F66E02030360718F09C012050D4
:1027E000324066E04030560710F0405056408F3F70
:1027F000910571F068F063E08030960710F48FEF78
:1028000007C064E08030960710F080E001C080953A
:1028100080832F3F310509F010F4822F0EC083E032
:102820002030380710F48FEF08C064E020303607FE
:1028300010F080E002C0822F80958C934F3F5105AD
:1028400009F010F4842F0EC083E04030580710F4D4
:102850008FEF08C064E04030560710F080E002C0FF
:10286000842F80958883DF91CF91089587FD80958F
:1028700090E080589F4F889F9001899F300D989FCE
:10288000300D1124232F3327AC01249FC001259F35
:10289000900D349F900D1124892F0895FB01DC01C8
:1028A00002C005900D9241505040D8F70895A0E025
:1028B000B0E0EDE5F4E10C949D147C01EB018A019C
:1028C000690109C0CE012196F6010995F7018193AE
:1028D0007F010150104001151105A1F7CDB7DEB7FA
:1028E000E8E00C94B914991B79E004C0991F96177D
:1028F00008F0961B881F7A95C9F780950895AA1B42
:10290000BB1B51E107C0AA1FBB1FA617B70710F0DA
:10291000A61BB70B881F991F5A95A9F7809590950C
:10292000BC01CD0108952F923F924F925F926F921A
:102930007F928F929F92AF92BF92CF92DF92EF924F
:10294000FF920F931F93CF93DF93CDB7DEB7CA1BD0
:10295000DB0B0FB6F894DEBF0FBECDBF09942A88FB
:10296000398848885F846E847D848C849B84AA84A3
:10297000B984C884DF80EE80FD800C811B81AA8130
:10298000B981CE0FD11D0FB6F894DEBF0FBECDBFFB
:08299000ED010895F894FFCF5A
:10299800010204080A1428500700200E0003002032
:1029A8000040008000000118000002000400080038
:1029B80010212230C2C180A1A250424121223024DC
:1029C800C180A144504241212210C2C180A1A21855
:0A29D8004241040503FFFFFFFF006A
:00000001FF
